:020000040001F9
:10B0000078210020D5B00100EFB00100F1B00100BF
:10B010000000000000000000000000000000000030
:10B02000000000000000000000000000F3B001007C
:10B030000000000000000000F5B00100F7B00100C2
:10B04000F9B00100F9B00100F9B00100F9B0010058
:10B05000F9B0010000000000F9B00100F9B00100F2
:10B06000F9B00100F9B00100F9B00100F9B0010038
:10B07000F9B00100F9B00100F9B00100F9B0010028
:10B08000F9B00100F9B00100F9B00100F9B0010018
:10B09000F9B00100F9B00100F9B00100F9B0010008
:10B0A000F9B00100F9B0010000000000000000004C
:10B0B0000000000000000000000000000000000090
:10B0C0000348854600F074F800480047B9B901000C
:10B0D000782100200321094802680A4302600848D9
:10B0E00002680A4302600748804707480047FEE7B6
:10B0F000FEE7FEE7FEE7FEE7FEE70000240500406E
:10B1000054050040C1B20100C1B0010003460B4329
:10B110009B0703D009E008C9121F08C0042AFAD20D
:10B1200003E00B780370401C491C521EF9D2704793
:10B13000421C0178401C0029FBD1801A704703464D
:10B140000A780270401C491C002AF9D11846704741
:10B15000F0B51FB40646002082B005464024019198
:10B1600000901BE0019922460F46304600F042F85D
:10B17000049A059B801A994110D31046194622461D
:10B1800000F028F8361A8F4101972246012000214D
:10B19000009F00F01FF838184D4100902046641EB3
:10B1A0000028DFDC019B00982946324607B0F0BD3D
:10B1B000064C0125064E05E0E36807CC2B430C3C0A
:10B1C00098471034B442F7D3FFF77EFF78BD0100F3
:10B1D00098BD010010B5202A04DB0146203A9140B9
:10B1E000002010BD914020239C1A0346E3401943E0
:10B1F000904010BD10B5202A04DB0846203AD0400C
:10B20000002110BD0B46D340D0402024A21A91400B
:10B210000843194610BD0000FFB5114F04463878A9
:10B2200081B01D461646002801D100F099F8386912
:10B23000A04211D918200A4960434118002C06D0B9
:10B240000298CE610D6288610020886248620A9887
:10B25000C862002005B0F0BD0020C043FAE700003E
:10B26000FC18002070B50E461821484313491446B7
:10B270004518E86A1835002804D001280FD00228A4
:10B2800005D113E0284600F0A1F8A04201D2002425
:10B2900011E022463146284600F0D3F80BE028465C
:10B2A00000F094F8A042F4D20446F2E73146284672
:10B2B00000F097F80446204670BD0000FC180020FE
:10B2C00010B500F055FB002805D01F491D48486007
:10B2D000C8131E4988611E48018CC9B201290BD1CF
:10B2E000828C120708D1028D1206120F042A03D194
:10B2F000828D1206120F0AD0012921D1818C0907F3
:10B300001ED1018D0906090F0A2904D007E0114A50
:10B3100001219160F5E7828D1206120F05D00D29EB
:10B320000ED1808D0006000F0AD10B48016801295B
:10B3300004D00A49016001680129FCD1C0214161A2
:10B3400010BD0000DFFF07C000050040006C00409A
:10B35000C00F00F00006004000EC064075930000AE
:10B3600010B5124C02202061606111A0A061134849
:10B37000E0610120800220620020A06260620CA1D6
:10B38000A1642146E0621039E16410212165A065C5
:10B390006065E0650AA1E01DFFF7D1FE09A1204626
:10B3A000FFF7CDFE2020A07110BD0000FC1800208A
:10B3B0005465726D696E616C00000000EC14002031
:10B3C0005254540053454747455200000269C16832
:10B3D0008A4203D88068401A801800E0501A401E44
:10B3E0007047F7B5064682B000200090F468174613
:10B3F0003069A04201D9051B02E0B168201A0D1A7C
:10B40000B0686D1E001BA84200D80546BD4200D39F
:10B410003D4670682A4600190399FFF777FE0098A9
:10B420007F1B401900900398641940190390B0687D
:10B43000A04200D10024F460002FD9D1009805B0BB
:10B44000F0BDF7B5C668174604468068851B60687E
:10B45000BD4206D980190199FFF758FEF019E06046
:10B46000FEBD2A4680190199FFF750FE01987E1B08
:10B47000411932466068FFF749FEE660FEBD0000F4
:10B480000FB410B504A9074B02AA039800F028F8DE
:10B49000044602A9002000F05DFA204610BC08BC5A
:10B4A00004B0184755B9010030B47446641E2578BD
:10B4B000641CAB4200D21D46635D5B00E31830BCE8
:10B4C000184702E008C8121F08C1002AFAD17047C5
:10B4D0007047002001E001C1121F002AFBD1704714
:10B4E000FFB591B00F460546002606E025280AD094
:10B4F000149A139990476D1C761C28780028F5D172
:10B50000304615B0F0BD002400940121F34A0294A6
:10B5100000E004436D1C2B780846203B9840104205
:10B52000F7D128782A280ED0022128780246303A0E
:10B53000092A15D8009A0A235A43303A80180C4336
:10B540006D1C0090F1E701CF0090002805DA012082
:10B5500040030443009840420090022004436D1CC5
:10B5600028782E2815D10420044368786D1C2A28D9
:10B570000AD101CF6D1C02900BE002990A225143BF
:10B58000303940186D1C029028780146303909295D
:10B59000F3D928786C2810D006DC4C281AD06828FB
:10B5A0000ED06A2817D104E0742813D07A2812D15B
:10B5B00010E00120400504430CE00121090501E0F1
:10B5C000032109050C436978814203D1012000055C
:10B5D00024186D1C6D1C287803906E281ED00CDC7E
:10B5E000632831D004DC00288AD0582811D1B2E079
:10B5F00064287BD069280CD178E073282DD004DC36
:10B600006F2870D0702804D1A7E075286CD07828F6
:10B610006BD0149A13999047761C62E06002400F39
:10B62000022807D003280AD0042838680AD0066008
:10B630003F1D56E03868F11706604160F8E738684A
:10B640000680F5E70670F3E738786946087400204D
:10B65000487404A80390012003E038680390002098
:10B66000C0433F1D61070FD5002101E00199491C2E
:10B67000029A0191914213DA8142F7DB019A039910
:10B68000895C0029F2D10BE0002101E00199491CFD
:10B6900001918142FADB019A0399895C0029F5D175
:10B6A00001990098139A401A00902146149B00F0CB
:10B6B0003BF901998019461807E00398039900782F
:10B6C000491C0391149A139990470198401E0190C8
:10B6D000401CF2D12146149B139A009800F014F9F3
:10B6E00086196D1C09E741E033E034E00A200021AF
:10B6F000049005916002410F022905D001CFC217C5
:10B700009446032905D007E0FF1DFF08FF0003CF83
:10B7100006E000B2C2179446042902D140B2C11714
:10B720008C4600226146944506DA0A4600214042D2
:10B7300091418C462D2102E0210504D52B216A463A
:10B740001176012103E0E10701D02021F7E7019103
:10B7500054E00A200BE0102009E0102004900021A2
:10B760000420044308200591029003E008200021F2
:10B77000059104906002410F022905D001CF0022FB
:10B780009446032906D006E0FF1DFF08FF0003CF03
:10B790008C4603E080B2042900D1C0B2002101919F
:10B7A00021072BD50399702906D0049A1021059BF7
:10B7B0004A401A4305D00EE040216A461176012125
:10B7C00008E06146014306D030216A4611760399AC
:10B7D000517602210191049A0821059B4A401A439F
:10B7E0000CD16146014301D1610707D530216A467A
:10B7F0001176012101910299491E0291039958295C
:10B8000004D037A103910FA90F910DE039A1F9E7F9
:10B810006146059B049AFFF79BFC039B8C469B5C4F
:10B820000F9A521E0F92137061460143F0D10F9888
:10B8300007A9081A20300390600704D501200004EE
:10B840008443029801E0012002900399884201DDBF
:10B85000401A00E000204118029001980918009851
:10B86000401A0090E00306D42146149B139A0098D6
:10B8700000F05AF886190020049008E006A9085C38
:10B88000149A139990470498401C761C04900199CF
:10B890008842F3DBE0030CD52146149B139A0098F1
:10B8A00000F042F8861904E0149A3020139990476A
:10B8B000761C0299481E02900029F5DC08E00F98DA
:10B8C0000F990078491C0F91149A13999047761C90
:10B8D0000399481E03900029F1DCFBE609280100CA
:10B8E00030313233343536373839616263646566F6
:10B8F00000000000303132333435363738394142B8
:10B900004344454600000000F8B5044600251E46A5
:10B910001746880404D405E039462020B0476D1C42
:10B92000641EF9D52846F8BDFFB50446002581B050
:10B930001E46C80301D5302700E02027880404D51F
:10B9400005E038460399B0476D1C641EF9D52846BA
:10B9500005B0F0BD0A68531C0B60107070470029D9
:10B9600001DA002070470268511801600120704719
:10B970001048018CC9B2012917D1818C090714D153
:10B98000018D09060A0F03D1828D1206120F0ED007
:10B99000090F012903D1828D1206120F07D0032946
:10B9A00003D1808D0006000F01D0002070470120D8
:10B9B00070470000C00F00F0002000F09BF91DA1AF
:10B9C000032000F083F9002003211D4A01252B46A6
:10B9D0008340DB011B0F02D083009B181960401CC1
:10B9E0002028F4D3174F184E00247A681748015DB9
:10B9F0002846884001469043B8601140F9602246CD
:10BA000013A1032000F068F9174A1849126830465C
:10BA100000BF00BF00BF00BF00BF00BF00BF00BF2E
:10BA20008A4200D000BF401EF2D1641C042CDCDB33
:10BA3000DAE700003A494E464F3A496E6974000011
:10BA4000000700500005005040420F0074BD010087
:10BA50003A494E464F3A0A4C6564206368616E6706
:10BA60006564202564000000CC1300200024F4004D
:10BA700000487047BDBA0100F8B50C4C0546207867
:10BA8000002804D06078854201D10020F8BD01264D
:10BA90003302074A07A100200096FFF7BDFB0028EC
:10BAA00001D00820F8BD26706570EEE7C8130020AD
:10BAB000D01300204E6F726D616C0000F0B5C3B002
:10BAC0001746084600224B990092499A1C46511885
:10BAD0000291002801D00A2100E0002103AE01916B
:10BAE000002C15D131466A4600F02CF900286AD0A6
:10BAF0003846FFF71DFBC22800D9C2200546009832
:10BB00002A4630183946FFF701FB0098401900908B
:10BB10000199009803AA41181018313151180022D8
:10BB200003E020230370401C521C019B9A42F8D36F
:10BB30000026029A944207D320220270427082703B
:10BB40000A70C01C491C26E0499A944202D2489AC5
:10BB5000125D02E0A31A4A9AD25C01259446AB001A
:10BB60006246DA4013071B0F092B01D9373300E077
:10BB7000303301277F1B6D1EC3556A1CEFD1202275
:10BB8000827062461346203BC01C5E2B00D92E22D9
:10BB90000A70491C641C761C102ECAD30D220A7030
:10BBA0000A224A7020210170009901980918433136
:10BBB00003A8009100F0AFF8002804D00020009006
:10BBC00002988442A4D3204643B0F0BDFFB5C5B06F
:10BBD0000846002505AE1C464E9F314604AA049532
:10BBE00000F0B0F800282FD03B00FFF75DFC070500
:10BBF000131A2F38434F21004798FFF799FA0499F9
:10BC000005464018FF2813D870182A464799FFF7B1
:10BC10007DFA0DE00498226830184799FFF730FC50
:10BC200005E004980CCC30184799FFF729FC05462D
:10BC3000294604A8FFF793FE002804D0FF200499AA
:10BC4000013081422ED9002049B0F0BDA06800909B
:10BC500004980CCC30184799FFF712FCE7E7E1682D
:10BC6000A0680090019104980CCC30184799FFF718
:10BC700007FCDCE72046083007C86B4607C304987A
:10BC80000CCC30184799FFF7FBFBD0E72046083073
:10BC90000FC86D460FC504980CCC30184799FFF7B4
:10BCA000EFFBC4E705A800F036F8CDE70048704781
:10BCB000CDBB010038B50093034B0D465C691346BC
:10BCC00000212A46A04738BDD014002010B500231B
:10BCD0001A46FFF7EFFF10BD08B5009201236A4630
:10BCE000FFF7E8FF08BD0000014A9161506170470D
:10BCF000D014002070B50120FFF7BEFE040008D16B
:10BD0000FFF7D4FF0546FFF7B3FE01462846FFF7CD
:10BD1000EBFF204670BDF8B50746012000250C4614
:10BD20000A260090791922460020FFF79BFA2D1869
:10BD3000241A002801D1761E01D0002CF2D10098DF
:10BD4000F8BD000010B5144602460120002A09D0B3
:10BD50000846126805A1FFF793FB01462046FFF74E
:10BD6000FEFD10BD0021216010BD00005B253038B4
:10BD7000645D00001516171898BD0100C813002057
:10BD800008000000C2B40100A0BD0100D0130020D3
:10BD9000A80D0000D2B40100000000000024F4004F
:040000050001B0C185
:00000001FF
